:020000040000FA
:1000000023015604FF0FFF0FFF0FFF0FFF0FFF0F1E
:10001000FF0FFF0FFF0FFF0FFF0FFF0FFF0FFF0F70
:10002000FF0FFF0FFF0FFF0FFF0FFF0FFF0FFF0F60
:10003000FF0FFF0FFF0FFF0FFF0FFF0FFF0FFF0F50
:10004000FF0FFF0FFF0FFF0FFF0FFF0FFF0FFF0F40
:10005000FF0FFF0FFF0FFF0FFF0FFF0FFF0FFF0F30
:10006000FF0FFF0FFF0FFF0FFF0FFF0FFF0FFF0F20
:10007000FF0FFF0FFF0FFF0FFF0FFF0FFF0FFF0F10
:10008000FF0FFF0FFF0FFF0FFF0FFF0FFF0FFF0F00
:10009000FF0FFF0FFF0FFF0FFF0FFF0FFF0FFF0FF0
:1000A000FF0FFF0FFF0FFF0FFF0FFF0FFF0FFF0FE0
:1000B000FF0FFF0FFF0FFF0FFF0FFF0FFF0FFF0FD0
:1000C000FF0FFF0FFF0FFF0FFF0FFF0FFF0FFF0FC0
:1000D000FF0FFF0FFF0FFF0FFF0FFF0FFF0FFF0FB0
:1000E000FF0FFF0FFF0FFF0FFF0FFF0FFF0FFF0FA0
:1000F000FF0FFF0FFF0FFF0FFF0FFF0FFF0FFF0F90
:10010000FF0FFF0FFF0FFF0FFF0FFF0FFF0FFF0F7F
:10011000FF0FFF0FFF0FFF0FFF0FFF0FFF0FFF0F6F
:10012000FF0FFF0FFF0FFF0FFF0FFF0FFF0FFF0F5F
:10013000FF0FFF0FFF0FFF0FFF0FFF0FFF0FFF0F4F
:10014000FF0FFF0FFF0FFF0FFF0FFF0FFF0FFF0F3F
:10015000FF0FFF0FFF0FFF0FFF0FFF0FFF0FFF0F2F
:10016000FF0FFF0FFF0FFF0FFF0FFF0FFF0FFF0F1F
:10017000FF0FFF0FFF0FFF0FFF0FFF0FFF0FFF0F0F
:10018000FF0FFF0FFF0FFF0FFF0FFF0FFF0FFF0FFF
:10019000FF0FFF0FFF0FFF0FFF0FFF0FFF0FFF0FEF
:1001A000FF0FFF0FFF0FFF0FFF0FFF0FFF0FFF0FDF
:1001B000FF0FFF0FFF0FFF0FFF0FFF0FFF0FFF0FCF
:1001C000FF0FFF0FFF0FFF0FFF0FFF0FFF0FFF0FBF
:1001D000FF0FFF0FFF0FFF0FFF0FFF0FFF0FFF0FAF
:1001E000FF0FFF0FFF0FFF0FFF0FFF0FFF0FFF0F9F
:0E01F000FF0FFF0FFF0FFF0FFF0F67059008B7
:020000040000FA
:021FFE001B00C6
:020000040000FA
:080200000100020003000400EC
:020000040000FA
:0201FE00000CF3
:00000001FF
